:100000000C94F8030C9415040C9415040C9415042A
:100010000C9415040C9415040C9415040C941504FC
:100020000C9415040C9415040C94B2250C9486269B
:100030000C94C9200C9415040C9415040C9415040C
:100040000C9415040C9415040C9415040C941504CC
:100050000C9415040C9450210C9415040C94150464
:100060000C9415040C9415040C9415040C941504AC
:100070000C9415040C9415040C9415040C9415049C
:100080000C9415040C9415040C9415040C9415048C
:100090000C9415040C9415040C9415040C9415047C
:1000A0000C9415040C9415040C9415040000000025
:1000B0000000000000000000000000000000000040
:1000C0000000000000000000000000000000000030
:1000D0000000000000000000000000000000000020
:1000E0000000000000000000000000000000000010
:1000F0000000000000000000000000000000000000
:1001000000000000000000000000000000000000EF
:10011000F0F0F0F0F0F0F0F0F0F0F0F0F0F0F0F0DF
:1001200000000000000000000000000000000000CF
:10013000000000000000000000000000F0F0F0F0FF
:10014000F0F0F0F0F0F0F0F0F0F0F0F0F0F0F0F0AF
:10015000F0F0F0F0F0F0F0F000000000000000001F
:10016000000000000000000000000000000000008F
:10017000000000000000000000000000000000007F
:1001800000000000F0F0F0F00F0F0F0F0F0F0F0F37
:10019000000000000000000000000000000000005F
:1001A0000F0F0F0FF0F0F0F000000000F0F0F0F093
:1001B0000F0F0F0FFFFFFFFFFFFFFFFFFFFFFFFF0F
:1001C000000000000000000000000000FFFFFFFF33
:1001D000F0F0F0F0F0F0F0F00F0F0F0F0F0F0F0F27
:1001E0000F0F0F0FF0F0F0F0F0F0F0F00000000053
:1001F00000000000000000000000000000000000FF
:10020000FFFFFFFF000000000000000000000000F2
:100210000F0F0F0FFFFFFFFF0F0F0F0F000000006A
:1002200000000000FFFFFFFF00000000F0F0F0F012
:100230000F0F0F0F00000000000000000000000082
:100240000F0F0F0FF0F0F0F00F0F0F0F0000000076
:1002500000000000000000000F0F0F0FF0F0F0F0A2
:100260000F0F0F0F00000000000000000F0F0F0F16
:10027000F0F0F0F00000000000000000FFFFFFFFC2
:10028000000000000000000000000000000000006E
:10029000000000000000000000000000000000005E
:1002A000F0F0F0F00F0F0F0F000000000000000052
:1002B0000F0F0F0FF0F0F0F0F0F0F0F0F0F0F0F0C2
:1002C0000F0F0F0F000000000F0F0F0FF0F0F0F0F6
:1002D000F0F0F0F0F0F0F0F0FFFFFFFFF0F0F0F0E2
:1002E000FFFFFFFFFFFFFFFFFFFFFFFF0F0F0F0FDE
:1002F0000F0F0F0F0F0F0F0F0F0F0F0FFFFFFFFF4E
:1003000000000000000000000000000000000000ED
:1003100000000000F0F0F0F0F0F0F0F00F0F0F0F21
:1003200000000000000000000000000000000000CD
:1003300000000000FFFFFFFF00000000FFFFFFFFC5
:1003400000000000000000000000000000000000AD
:100350000F0F0F0FF0F0F0F0F0F0F0F0FFFFFFFFE5
:100360000F0F0F0F00000000000000000000000051
:100370000000000000000000FFFFFFFF0000000081
:10038000000000000000000000000000F0F0F0F0AD
:100390000F0F0F0F00000000000000000000000021
:1003A000000000000000000000000000FFFFFFFF51
:1003B000FFFFFFFFFFFFFFFFFFFFFFFFFFFFFFFF4D
:1003C000FFFFFFFFFFFFFFFFFFFFFFFFFFFFFFFF3D
:1003D000FFFFFFFF0F0F0F0F0F0F0F0F00000000A9
:1003E0000000000000000000F0F0F0F0F0F0F0F08D
:1003F0000F0F0F0F0F0F0F0F000000000000000085
:1004000000000000F0F0F0F0FFFFFFFF0000000030
:1004100000000000000000000000000000000000DC
:1004200000000000000000000000000000000000CC
:1004300000000000000000000000000000000000BC
:1004400000000000000000000000000000000000AC
:10045000000000000000000000000000F0F0F0F0DC
:10046000F0F0F0F00F0F0F0FF0F0F0F0F0F0F0F010
:100470000000000000000000F0F0F0F0F0F0F0F0FC
:100480000F0F0F0FFFFFFFFF000000000000000034
:10049000000000000000000000000000000000005C
:1004A0000000000000000000000000001E001F000F
:1004B0002000210022002300240025001E0F05003B
:1004C000047F3F1F643214643214783C1E1E140AE9
:1004D000052223252628292A2C2D2F303233353684
:1004E000383A3B3D3E4042434547494A4C4E5051C5
:1004F000535557595A5C5E6062646668696B6D6FEC
:1005000071737577797B7D7F81838587898A8C8EEE
:1005100090929496989A9C9E9FA1A3A5A7A8AAACF6
:10052000AEAFB1B3B4B6B8B9BBBCBEBFC1C2C3C530
:10053000C6C7C9CACBCCCDCED0D1D2D2D3D4D5D6D2
:10054000D7D7D8D9D9DADADBDBDBDCDCDCDCDCDD05
:10055000DDDDDDDCDCDCDCDCDBDBDBDADAD9D9D8E9
:10056000D7D7D6D5D4D3D2D2D1D0CECDCCCBCAC981
:10057000C7C6C5C3C2C1BFBEBCBBB9B8B6B4B3B1B0
:10058000AFAEACAAA8A7A5A3A19F9E9C9A9896944B
:1005900092908E8C8A89878583817F7D7B79777520
:1005A00073716F6D6B6968666462605E5C5A5957FF
:1005B000555351504E4C4A4947454342403E3D3BBE
:1005C0003A3836353332302F2D2C2A292826252348
:1005D00022FFAA7F55400001010101010101010133
:1005E00002020202020202020203030303030303E4
:1005F00003040404040404040505050505060606B1
:100600000606070707070708080808090909090A6D
:100610000A0A0B0B0B0C0C0C0D0D0D0E0E0E0F0F12
:100620000F101011111112121313141415151616A0
:100630001717181819191A1A1B1B1C1D1D1E1E1F0F
:100640002020212222232424252626272829292A5E
:100650002B2C2D2D2E2F3031323233343536373886
:10066000393A3B3C3D3E3F40414243444546474882
:10067000494A4C4D4E4F50515354555658595A5B58
:100680005D5E5F616264656668696B6C6D6F7072F8
:10069000737577787A7B7D7E8082838587888A8C64
:1006A0008E8F91939596989A9C9EA0A2A3A5A7A998
:1006B000ABADAFB1B3B5B7BABCBEC0C2C4C6C9CB8F
:1006C000CDCFD1D4D6D8DBDDDFE2E4E7E9EBEEF045
:1006D000F3F5F8FAFDFF00AE00AF00DA128180D921
:1006E000F1DB20A4A62EAF00A0C000A1C800AED5AB
:1006F00080A83FD300408D142000120354007500E1
:10070000740065006C0050006100640000001C0370
:1007100049007400730046006900720065006D00B6
:1007200061006E00530061006D00000004030904C5
:1007300009023B00020100A0FA09040000010301C4
:100740000100092111010001224000070581030871
:10075000000109040100010300000009211101004A
:10076000012232000705820320000112010002006D
:1007700000000800CB9FF001000102000105010903
:1007800080A101850319012AB700150126B700953C
:100790000175108100C0050C0901A1018504190132
:1007A0002AA002150126A002950175108100C0053E
:1007B000010906A101050719E029E71500250195A2
:1007C0000875018102950175088101050719002945
:1007D000FF150026FF009506750881000508190120
:1007E0002905950575019102950175039101C000D8
:1007F00011241FBECFEFDAE0DEBFCDBF11E0A0E0D5
:10080000B1E0EEEDF3E502C005900D92A23DB10717
:10081000D9F726E0A2EDB1E001C01D92AE3EB207CD
:10082000E1F70E944D120C94D7290C94000082E04D
:1008300008950E947A1C882331F060E074E08CEA0D
:1008400090E00E94041B80E0089581E0089581E01B
:1008500008950E942704089508950E942C04089585
:10086000A5E0B0E0E6E3F4E00C94C92849835A839C
:100870003091D90189819A81311119C0662399F08B
:10088000222389F00E94A309182F682F89819A8159
:100890000E94800969817A81812F0E941210259619
:1008A000E3E00C94E5280E949109182FF3CF0E94F1
:1008B000A30969817A81F1CFFC01262F4081518102
:1008C0006281738184810E943004089581E00895DB
:1008D000CF93DF93EC0160E00E945C04BE010E94B4
:1008E0002D04DF91CF9108950E94541108950E9424
:1008F0005811089508950E944B080E947A042FEF22
:1009000084E39CE0215080409040E1F700C000006B
:1009100008950E947B040E94742108950E947B0424
:100920000E94852108950F931F93CF93DF938C012D
:1009300061E00E945C04EC01B8010E94290481116D
:1009400006C080E0DF91CF911F910F910895B8010B
:10095000CE010E94A21E8823A1F3B801CE010E94FD
:10096000A61C882371F3B801CE010E94141E8823AF
:1009700041F3B801CE010E946F19882311F3F801E9
:100980008281882361F0CB35FDE5DF0701F158F462
:10099000C115ECE5DE0791F0CF3DDC4591F0C801D3
:1009A0000E942504CFCFCD358DE5D80769F090F0B2
:1009B000C83ADD45A1F70E948E04C3CF0E94890486
:1009C000C0CF0E945D0EF7CF0E949B0DE8CF0E9422
:1009D000A50DE5CF0E94A90DE2CF0E94A5200E949F
:1009E00010050E94D5170E945F1C08950E941405EF
:1009F0000E94AC180E94AA20089508950E94FD0448
:100A0000089581E008950E94010508950895CF9307
:100A1000C82F0E94FE048C2F0E940305CF910895D9
:100A200080E00E94070508950E94EA1F0E940705C2
:100A30000895CF930E94EA1FC82F8091D4018C178C
:100A400079F0C093D4010E9435216093D501709351
:100A5000D6018093D7019093D8018C2F0E9407056F
:100A6000CF910895ABE0B0E0E8E3F5E00C94CA283C
:100A70004F83588769877A878B8761110E94E60CBC
:100A80001E821D8285E0FE013796DE0111960190DF
:100A90000D928A95E1F78C819D81892B61F44981C2
:100AA0005A816B817C818D819E810E940F0C2B96D7
:100AB000E2E00C94E62889819A8189238F3F79F3BB
:100AC000CE0101960E9466048111E9CFF0CFFC01AE
:100AD000808191810E94D5090895CF93C82F8823E2
:100AE000B9F08CEF8C0F813AA8F46C2F809104013F
:100AF000909105010E944020882329F08C2F0E94AC
:100B0000A60C0E94070D8C2F0E949E0C0E94070DC0
:100B1000CF91089580E28C0F883048F4C77081E04F
:100B200001C0880FCA95EAF70E94C90CEFCFEBE528
:100B3000EC0FE33040F4F0E0E55AFE4F808190E0A6
:100B40000E940220E5CFC85AC73110F7EC2FF0E021
:100B5000EE0FFF1FE35DFE4F808191810E94182000
:100B6000D7CF882339F19CEF980F913A28F40E944F
:100B7000A60C0E94070D089590E2980F983050F44B
:100B8000877091E001C0990F8A95EAF7892F0E943A
:100B9000CF0CEFCF9BE5980F933028F490E080E0E6
:100BA0000E9402200895885A873120F490E080E066
:100BB0000E94182008951F93CF93DF93182FEB0105
:100BC0000E946D05209739F4812F0E94B105DF91B5
:100BD000CF911F9108958FE99FE00197F1F700C031
:100BE00000002197EFCF70E060E0893311F460E5F9
:100BF00070E00E94DB050895882321F00E94C90C53
:100C00000E94070D0895882321F00E94CF0C0E94B6
:100C1000070D0895B0E0A0E0E0E1F6E00C94C328F1
:100C20006C01D62FC72FFC011281F580F2949FE052
:100C3000F9220E94BF0CE82E8823B9F0E12E11237F
:100C4000A1F08C2F807F803421F080E28D0F8830DE
:100C5000D0F08091C10282FF16C082E00E946A0D2E
:100C60000E94BF0C91E0E82EE926BC2EB2948FE0E2
:100C7000B822FBE0FB1508F468C0EB2DF0E0E7526A
:100C8000F64D0C948328E12CF0CF0C2F0F70C07F11
:100C900011F00295007F112399F0002359F080E2B2
:100CA0008D0F883010F0D11107C0802F0E94C90C21
:100CB0000E94070D8D2F41C0802F0E94D90CF8CFC4
:100CC0008D2F0E94B105002309F43FC080E28D0FF3
:100CD000883010F0D11104C0802F0E94CF0C03C0C7
:100CE000802F0E94DF0C0E94070D2FC00C2F0F7069
:100CF000C07FC03211F00295007FDD2381F0D1303A
:100D000009F463C0112309F46DC0FF2009F463C026
:100D1000F601858180FFCECF8F7085835CC0809186
:100D2000C10282FD33C0112359F0002329F0802F26
:100D30000E94C90C0E94070D80E00E946D0505C04D
:100D400080E00E94B1050111C7CFEB2DE850FF0BE9
:100D5000349720F40E94EA1F0E940705EE2089F0D4
:100D60000E94BB0C80FD0DC0F60112820E94B50CE2
:100D70000E94DE08C6010E940F080E94B50C0E9466
:100D8000EE08CDB7DEB7E9E00C94DF28112389F037
:100D9000F11006C00E94E90C802B0E94FC05D5CF03
:100DA00021E0F212F7CF0E94E90C802B0E94F00C98
:100DB000CCCFF11006C00E94FD0C802F0E940306CC
:100DC000C4CF31E0F31609F2F6CF112331F085E0FC
:100DD0008F1508F4BACF802FE0CF94E09F1508F468
:100DE000B4CFEBCFFF2049F3D93349F4FFEF27EE1F
:100DF00033E0F15020403040E1F700C000008D2F7B
:100E00000E94B105A2CF8C2F86958695837069F0DC
:100E1000813009F09ACF8D2F9C2F9370111102C051
:100E200090E080E00E94182090CF8D2F9C2F93702F
:100E3000111102C090E080E00E94022086CF8C2F2A
:100E40008370A1F5111181CF4D2F429546954770C2
:100E5000440F440F2D2F2F7030E0042E02C0220FBC
:100E6000331F0A94E2F790E080E0D4FF09C08FE0DE
:100E700090E002C0880F991F4A95E2F780959095FF
:100E8000C695C695C370822B932BC23049F058F497
:100E9000C13019F00E94AC0858CF0E94A30855CF6A
:100EA0000E94B50852CF0E94A0084FCF869511230B
:100EB00011F08C2F8170882309F447CF4D2F429574
:100EC00046954770440F440F2D2F2F7030E0042EAD
:100ED00002C0220F331F0A94E2F790E080E0D4FFB3
:100EE00009C08FE090E002C0880F991F4A95E2F791
:100EF00080959095C695C695C370822B932BC23072
:100F000049F058F4C13019F00E9419091ECF0E940F
:100F100010091BCF0E94220918CF0E94C40815CFC8
:100F2000CF70112329F08C2F0E94DE088D2F35CF32
:100F30008D2F0E9403068C2F0E94EE0806CFD23F11
:100F400051F160F4D03FB9F0D13F81F0112309F4A1
:100F500049C0F110AFCE8C2F8F7121C0D33F11F15A
:100F6000D43FA1F78091C10282FD26C08C2F8F71E2
:100F7000112311F314C0112349F084E08F1508F4F4
:100F8000E4CE8C2F8F710E940009DFCE95E09F1573
:100F900008F4DBCEF6CF8C2F8F711111CDCF0E94CC
:100FA000DE08D3CE112329F08C2F8F710E94D20836
:100FB000CCCE0E94CD08C9CE112349F0CF718C2F21
:100FC0000E94DE0863E08C2F0E944C0DBECE81E0B3
:100FD0000E946A0DE1E0EF1508F0B7CE82E00E94B2
:100FE0006A0DB3CEF11000CF8C2F8F71A5CF0F9368
:100FF0001F93CF93DF93EC01688179818A810E94EE
:10100000E0098C010E942B090E949F08B801CE01C3
:101010000E940A06DF91CF911F910F910895CF93FF
:10102000DF93EC018B819C81892B29F08881998148
:1010300089238F3F51F4DF91CF910895CE010E9413
:10104000F707CE010E946804F6CFCE010E949304F8
:101050008111F4CF0E94BF0C882369F38A81882311
:1010600051F38091C10282FFE6CF82E00E946A0DB7
:10107000E2CF90E080E00E94022090E080E00E94B9
:1010800018200E94E60C0E94070D08950E94AE0CE5
:101090000E94390808950E94D60C0E9446080895BF
:1010A00092959F70963091F058F4925F9F709230B5
:1010B00058F4803F19F030F4883E30F481E0089510
:1010C0009A5FF4CF843FD1F380E00895883EB0F377
:1010D000813FD1F7F3CFFC0183819481892B29F0E3
:1010E0008081918189238F3F11F480E00895808170
:1010F00091810E94D5090E9450080895A5E0B0E0B2
:10110000E4E8F8E00C94CA282596E2E00C94E6287E
:10111000A6E0B0E0EEE8F8E00C94CA282696E2E0FB
:101120000C94E62808950E94920808950E9493085E
:101130009093E1018093E0010E9439080895089599
:101140000E94960808952091E0013091E101822BE0
:10115000932B0E94960808952091E0013091E101BF
:10116000822393230E94960808952091E0013091F4
:10117000E101822793270E94960808950E94920811
:1011800008950E94BE0808950E94C1089093DF014F
:101190008093DE010E943908089590E080E00E946B
:1011A000C408089521E030E0A90102C0440F551F92
:1011B0008A95E2F7CA010E94C408089521E030E050
:1011C00002C0220F331F8A95E2F78091DE019091D1
:1011D000DF01822B932B0E94C408089521E030E0A8
:1011E00002C0220F331F8A95E2F720953095809137
:1011F000DE019091DF01822393230E94C4080895A9
:1012000021E030E002C0220F331F8A95E2F780917F
:10121000DE019091DF01822793270E94C408089580
:101220002091DE013091DF01822B932B0E94C408B4
:1012300008952091DE013091DF01822393230E94E3
:10124000C40808952091DE013091DF0182279327A1
:101250000E94C40808950895262F277091E001C0C8
:10126000990F2A95EAF723E0769567952A95E1F795
:10127000660F771F660F771FFA01E60FF71F50E022
:1012800040E0682F70E08191DF0111979B01042EEF
:1012900002C0369527950A94E2F7217021952827F8
:1012A000292328272C934F5F5F4F4430510559F76E
:1012B0000895A82FA77023E0969587952A95E1F7C2
:1012C000880F991F880F991FFB01E80FF91F50E045
:1012D00040E080E0219130E00A2E02C0369527954B
:1012E0000A94E2F721703327042E01C0220F0A94DA
:1012F000EAF7822B4F5F5F4F4430510559F708954D
:10130000262F923068F4843058F434E0939FB00173
:101310001124680F711D4AED51E0822F0E942C09A3
:101320000895923070F4843060F444E0949F90010A
:1013300011246AED71E0820F932F911D0E945909CB
:10134000089580E00895B0E0A0E0E9EAF9E00C94A7
:10135000C3287C010091DE011091DF018091E00142
:101360009091E101082B192BCFE0D0E0CC24C3945D
:10137000D12CBC2EC6010C2E02C0880F991F0A94D6
:10138000E2F780239123892B49F4219790F7B12C20
:101390008B2DCDB7DEB7E9E00C94DF28B7018C2F99
:1013A0000E942C10019789F3F3CFCF93DF93EC01C8
:1013B0000E94A309BE010E942C10DF91CF910895D5
:1013C0001F93CF93DF93EB019091D901992339F0CB
:1013D000CB010E94D509DF91CF911F9108958823F9
:1013E00069F0CB010E94A309182F682FCE010E943B
:1013F0008009BE01812F0E942C10EDCFCB010E94ED
:101400009109182FF6CF1F93CF93DF93C091E2017C
:1014100016E08091E3018C1304C0DF91CF911F91FE
:101420000895D0E01C9FF0011D9FF00D1124EC5198
:10143000FE4F4081518162817381848195810E9438
:1014400088082196C770E5CF40911402509115028B
:101450006091160270911702809118029091190202
:101460000E94880808951F93CF93DF9380911902FB
:10147000807F09F049C080911602882309F444C096
:101480008091E201C091E301609114027091150214
:10149000A0911702B0911802D62FD72316E0C817D3
:1014A00099F190E0109711F0DF3F19F401968770E1
:1014B000F6CF189F9001199F300D1124F901EC51BE
:1014C000FE4F41814713F2CF40814613EFCF428157
:1014D0004111ECCF438154814A1B5B0B483C5105C1
:1014E00028F7809119028F70806180931902F901A9
:1014F000E751FE4F80818F708061808384E192E0AC
:101500000E940F080E94030ADF91CF911F91089556
:10151000A1E1B0E0EEE8FAE00C94C2288C0185E08D
:10152000F801DE011D9601900D928A95E1F7F80110
:10153000E28084E1C82E82E0D82E6091170270917B
:1015400018026115710509F44EC1909114022091A1
:101550001502892F82238F3F09F445C140815181B3
:10156000A380B480F0901602F501E61BF70BFF2074
:1015700009F4EAC080911902382F307FE83CF10568
:1015800008F0A3C031116DC0FE2C251316C09413B2
:1015900014C0E11012C08F708061809319020E9404
:1015A000240AC6010E940F0880911902F801858360
:1015B0008F2D6196EAE00C94DE28A114B10429F085
:1015C000842F85238F3F09F027C180E0F82FF17029
:1015D000DF2E80FF3CC08091E2012091E30136E0E4
:1015E000821315C04D875E878D859E850E94D50923
:1015F000292F22952F702230F0F0243018F59F709B
:10160000F1F0F8019581907FD1F4D12C1EC090E0CB
:10161000389FF001399FF00D1124EC51FE4F61818C
:10162000651306C06081641303C06281E6120FC0B7
:1016300001968770D5CF9F7011F0882331F3805EBB
:10164000883018F3C8010E940F08FD2CB1CFEE209E
:1016500009F4AECF80911902816080931902F12CB8
:10166000A7CF251306C0941304C0F801EE2009F497
:1016700087C0C8010E946B08882319F1EE2009F188
:1016800080911902803270F020911402309115027D
:1016900038872F831986BB86AA868C87CE0107964A
:1016A0000E940F0886E0F801A4E1B2E001900D92DB
:1016B0008A95E1F70E94330A0E94240AFF24F394DA
:1016C00077CFC8010E940F08F9CF311113C07A2DCE
:1016D000B98AA88A6E2D89890E947E0884E192E0E9
:1016E0000E940F0886E0F60111928A95E9F70E94A0
:1016F000240AB5CF25130FC094130DC0E1100BC001
:10170000F8018583C8010E940F0886E0F601119256
:101710008A95E9F74DCFC8010E946B08882389F2AA
:10172000EE2079F280911902803208F4BBCF20912B
:101730001402309115023A8329831B82BD82AC8248
:101740008E83CE010196ACCFE83CF10508F03EC097
:10175000FE2CEE2009F4B5CF25132AC0941328C01F
:101760008091190280FD1BC0982F907FC1F0F80175
:101770008583903F31F0982F907F905F8F70892BF9
:101780008583C8010E940F0886E0F801A4E1B2E059
:1017900001900D928A95E1F70E94240A09CF86E014
:1017A000F801A4E1B2E001900D928A95E1F700CF33
:1017B000C8010E946B08811175CF80911902816068
:1017C00080931902C8010E940F08F2CE7A2DB98ABF
:1017D000A88A6E2D89890E947E0886E0F601119202
:1017E0008A95E9F7D9CFEE2009F46BCFC8010E94A2
:1017F0006B08F82E882309F464CF86E0F801A4E191
:10180000B2E001900D928A95E1F784E192E00E94A6
:1018100067050E94330AC0CF81E08E25D7CEACE0A9
:10182000B0E0E5E1FCE00C94C9284F835887698754
:101830007A878B879C87CE0107960E94880A882327
:1018400069F08A859B85892B39F04F815885842FD3
:1018500085238F3F09F06BC016E05FC086E0FE0174
:101860003796DE01119601900D928A95E1F78A85EF
:101870009B85892B89F38F81988589238F3F61F31D
:101880002091E30130E0C9010196877099274091CA
:10189000E2014817190671F40E944B081092E30107
:1018A0001092E20186E0E4E1F2E0DF011D928A9508
:1018B000E9F7D2CF96E0929FD001939FB00D11240B
:1018C000AC51BE4FFE01319601900D929A95E1F711
:1018D0008093E3010E94030ABFCF819FC0011124BE
:1018E0008C519E4F0E94880A8823E9F0E091E20122
:1018F0001E9FF0011124EC51FE4F40815181628105
:101900007381848195810E9488088091E20190E032
:101910000196877099278093E2018091E20190916E
:10192000E3018913DACF2C96E3E00C94E52869856E
:101930007A858B859C850E9488088ECF682F809140
:101940000401909105010E9476200895682F8091EE
:101950000401909105010E9479200895809104016D
:10196000909105010E947C20089580912202859526
:1019700085958595089580912202877008959091AC
:101980002202977081E009F480E0089580912D0291
:10199000089590912D02892B80932D0208958095B2
:1019A00090912D02982390932D02089510922D026C
:1019B000089590912C02892B80932C020895809594
:1019C00090912C02982390932C02089510922C024F
:1019D000089580912302089508950E94EC0C0895C3
:1019E0009091C10292FF08C090912302981721F0B4
:1019F000809323020E94ED0C089580912302882396
:101A000029F01092230280E00E94ED0C0895CF93FC
:101A1000DF93E0910401F091050180912D02808314
:101A2000E0910401F0910501808190912C02892BB5
:101A3000808390912302992381F0E0910401F09139
:101A400005018081892B808380910401909105019B
:101A50000E942E2081110E94FD0CC0910401D091A2
:101A6000050148E050E06AE172E0CE010E945A2987
:101A7000892B59F088E0FE01AAE1B2E001900D92B5
:101A80008A95E1F7CE010E94F71FDF91CF9108956B
:101A900008950E94480D08959091C10292FF11C0CF
:101AA00098E0899F90011124622B609322020E948A
:101AB000DE08809122028595859585950E94490DC5
:101AC00008950E94DE0808951092220280E00E948C
:101AD000490D0895909122028095892380932202D6
:101AE000282F277091F4282F082E000C330B921703
:101AF000130659F09091C10292FF07C08595859514
:101B000085950E94EE080E94640D08959091C1028F
:101B100092FB222720F9281769F080FB92F9909315
:101B2000C1028091C0029091C1020E94D70D82E053
:101B30000E946A0D08958091C10282FB882780F976
:101B400091E089270E94860D089581E00E94860D0C
:101B5000089580E00E94860D08956FEF7FEF90E07A
:101B600080E00E94A229089590E080E00E947E29F2
:101B700021E0883E9E4F09F020E0822F089582E008
:101B800090E00E947029089583E090E00E947029FF
:101B90000895CF9384E090E00E947029C82F82E2DC
:101BA00090E00E947029982F8C2FCF910895CF93A9
:101BB000C92F682F84E090E00E9484296C2F82E274
:101BC00090E00E948429CF910895AB01BC018FE081
:101BD00090E00E9496290895AB01BC0183E190E05A
:101BE0000E949629089560E070E0CB010E94EC0D00
:101BF000089560E070E0CB010E94E50D0E94F30DB6
:101C0000089568EE7EEF90E080E00E94A22960E0F7
:101C100082E090E00E94842960E083E090E00E94EE
:101C200084291092E1011092E00160E084E090E0EC
:101C30000E94842964E082E290E00E94842960E0AE
:101C400085E090E00E94842960E086E090E00E94B8
:101C500084296FEF87E090E00E94842940E050E003
:101C6000BA0188E090E00E94962960E08DE090E063
:101C70000E94842940E050E0BA0188E190E00E948F
:101C8000962960E087E190E00E94842940E050E0DE
:101C9000BA018CE190E00E94962970E060E080E259
:101CA00090E00E94A22940E050E0BA0188E190E073
:101CB0000E9496290E94F90D08950E94010E089530
:101CC000682F8EE090E00E94842908950E943521BB
:101CD00060933602709337028093380290933902F2
:101CE00060933202709333028093340290933502F2
:101CF0000895089508950E947A0E089508950E9407
:101D00007E0E089586E191E10E94E01F0E94790E07
:101D10000E947B0E089581E008950E948B0E089525
:101D2000089508950E94900E0E94910E08950E94B9
:101D300035110E94060508950E9420210E94BB11C2
:101D40000E94970E80E00E94A51A0E9470180E94BF
:101D50007F0E0895AAE0B0E0E0EBFEE00C94C2280C
:101D60000E94CB111091300280E00E945B11181389
:101D700033C01091310281E00E945B1118132CC016
:101D80000E9429218C0180912E0290912F02081728
:101D90001907A1F08FEF89838A831B820E94292172
:101DA0008160782F9D838C8349815A816B818D81DD
:101DB0000E94320510932F0200932E0210E00E9421
:101DC000B6180E947C1C11110E94441B0E94190528
:101DD0002A96EAE00C94DE2880913A0281FD0E9466
:101DE00061110E948D0EC82E80E3A82E82E0B82ECD
:101DF00010E0812F0E945B11082FF50181915F0196
:101E0000081731F1D02ED826F12CEE24E3948E2D34
:101E10008D21B1F0CC20A1F0FE821F8391E08E2DA8
:101E2000802309F490E098870E9429218160782F0F
:101E30009A8789874E815F8168858A850E943205ED
:101E4000F394EE0CF4E0FF12E2CFF501319700833A
:101E5000113021F40E94660E11E0B1CF11E0C9CF1C
:101E6000CF93DF930E943110EC01811522E5920798
:101E7000E8F5811531E5930708F0A3C0883E910588
:101E800010F5803E910570F5883A910570F4853A19
:101E9000910508F078C08130910521F1009711F18A
:101EA000049700F5D0E0C0E01DC08F3B9105D0F74E
:101EB000C85AD0E0CC0FDD1FC25ADE4F0990D8813E
:101EC000C02DD4640FC0811540E5940708F066C0AA
:101ED000C11580E4D80708F05EC0CE019A9581153F
:101EE0009F4100F7CE01DF91CF910895811536E52E
:101EF000930718F5811545E5940708F07BC0C115D7
:101F000084E5D80708F071C09E01237033279C2F09
:101F100096959695C115D34508F458C0C1E0D0E018
:101F200002C0CC0FDD1F2A95E2F730E2939FC0017B
:101F30001124C82BD92BDA68D5CFC1158AE5D8076B
:101F400078F4C11529E5D20708F05EC0C11538E55F
:101F5000D30708F4A7CFDC2FCC27C06FD06AC2CF3D
:101F6000CE0190568115904208F09CCF8D2F8F7135
:101F70000E94D31090E0982F882788279F719C019A
:101F80002C2BE9013FC0C55AD0E0C457DE4FC881B1
:101F9000D0E0D064A7CFDF70D06AA4CF8370992738
:101FA00021E030E002C0220F331F8A95E2F7C69588
:101FB000C69580E2C89FE0011124C22BD32BDD68B7
:101FC00091CFD82FCC27C16FD06A8CCFC1E0D0E0A1
:101FD00002C0CC0FDD1F2A95E2F720E2929FC001DC
:101FE0001124C82BD92BDC687DCFDC2FCC27C46F04
:101FF000D06A78CF0E94D310C82FD0E0DC2FCC2736
:10200000CC27DF71D0626ECF8C2F8F700E94D310DF
:1020100034E0D695C7953A95E1F7CF709C2FEC0147
:10202000D06960CF7230A8F4643098F4E82FF0E003
:10203000EE0FFF1FE70FF11DEE0FFF1FEE0FFF1F4B
:10204000E60FF11DEE0FFF1FE455FB4F85919491B4
:10205000089580E090E008950E9412100E94300FD1
:10206000089582389105B9F1B0F48133910509F4EE
:102070007DC048F48932910509F46DC08A3291051A
:1020800009F47BC008958533910509F45FC0893355
:10209000910509F10895833E9105D9F138F4803E08
:1020A000910529F1823E910579F10895863E9105C9
:1020B000D9F1873E910509F43EC0843E910541F572
:1020C0002091C10221FF24C08091C00284FD19C06B
:1020D00087EE90E008952091C002237009F05AC065
:1020E0002091C10223FF14C089E290E0089520915D
:1020F000C00220FD38C03091C10230FF09C024FF6A
:1021000043C090E080E008952091C00222FDF7CF07
:1021100008952091C00222FD3AC03091C10230FDE5
:1021200039C024FFF5CFEDCF2091C00223FFF0CFBF
:1021300024FDE7CFCDCF2091C00223FD2EC03091EA
:10214000C10231FFEECF84EE90E008952091C002ED
:1021500025FFDECFC9CF2091C00225FD21C02091EF
:10216000C10223FFD5CF89E390E0D2CF2091C002F6
:1021700026FFCECF8AE290E008952091C00226FF8C
:10218000C7CF81E390E0089583EE90E0089582EE5A
:1021900090E0089580EE90E0089586EE90E0089536
:1021A00085E390E008959091C00292FF06C0282F29
:1021B00028712830F9F4877F846093FF06C0282FA8
:1021C00028712831F1F4877E84612091C10220FFBB
:1021D00006C0382F38713830D9F4877F816021FFED
:1021E00006C0282F28712831D1F4877E816194FDA3
:1021F000877E0895282F24712430F9F68B7F88601C
:10220000DCCF282F2471243101F78B7E8861DDCF4C
:10221000382F3171313019F78E7F8860E0CF282F49
:102220002171213121F78E7E8861E1CF80E0089510
:102230000E94AD0D08950E94CB112FEF86E791E02B
:10224000215080409040E1F700C000000E94CB1177
:1022500081E00E945B1180FF04C00E9418110E945F
:10226000742108950E941B1108950E94B40D8111DC
:1022700002C00E945D0E0E94BF0D80933A020E9430
:10228000C90D9093C1028093C0020E9432110E9436
:10229000C40D90E00E94A0088091DE019091DF01C2
:1022A0000E94C108089508950E9453110895089549
:1022B0000E9457110895E82FF0E0EC53FD4F808104
:1022C000089508951F93CF93DF932FE831E0C1E085
:1022D000D0E0D90150E040E08D918F3F91F0E82FA0
:1022E000E295EF70F0E011A18F70BE0101C0660FA2
:1022F0008A95EAF7962F9095912391A382A1862B38
:1023000082A34F5F5F4F4430510531F72C5F3F4F41
:1023100081E027393807E9F6DF91CF911F910895C1
:10232000CF93DF93AC0170E0FB01EE0FFF1FEE0FC8
:10233000FF1FE157FE4FA4E0B1E080E091919F3F85
:1023400081F0C92FC295CF70D0E028A130E09F70F6
:1023500002C0359527959A95E2F79B2F20FD90E0D6
:10236000892BBB0FA15051F7640F751FFB018083B0
:10237000DF91CF9108950E9462111092C5021092D0
:10238000C4021092C3021092C20282E00E940112A3
:102390000E9474040895A2E0B0E0E1EDF1E10C9434
:1023A000C9281A82198260E0CE0101960E9490111C
:1023B00061E0CE0101960E94901142E050E0BE0122
:1023C0006F5F7F4F82EC92E00E945A2921E00097D4
:1023D00009F420E0892B31F089819A819093C3021E
:1023E0008093C20242E064EC72E082EC92E00E94D0
:1023F0000212182F0E947704812F2296E3E00C949A
:10240000E5280895CF92DF92EF92FF920F931F93EA
:10241000CF936C017B01042F222349F081E080934C
:102420003D020E94292190933C0280933B02C0917F
:102430003D02C1110AC0C0E08C2FCF911F910F91B6
:10244000FF90EF90DF90CF90089580913B029091A4
:102450003C020E944121059770F310E0A801B601EB
:10246000C7010E945A29892B41F0A801B601C70172
:102470000E94672910923D02DFCFC0E0FBCF0E948F
:1024800008230E949C0E0E94152308950E941A237F
:102490000E94AA0E0E94342308950E94C2200E9426
:1024A000EE220E94820E0E943F120E9446120E945B
:1024B000920EFBCFEF92FF920F931F93CF93DF9378
:1024C000EB01E82FD1110EC0442321F0F0E0EA52D5
:1024D000FA4FE4916E2F7E2F8E2FCDB7DEB7E6E058
:1024E0000C94E2280D2F10E0282F30E0442329F02F
:1024F0002A523A4FF901249130E0F6E0CF9FC00113
:102500001124EFEFF0E0BF010E943928AB018C2FBE
:1025100090E0880F991FA5E5A49FB001A59F700DBD
:102520001124861B970B982F990F980FBF01601BE2
:10253000710B629FD001639FB00D729FB00D11248B
:102540008B2F9D9FB0011124672F7727EF01C61BAA
:10255000D70BBE01629FE001639FD00D729FD00D2B
:1025600011247F01E91AF108E09EB001E19E700D8F
:10257000F09E700D1124672F7727E61BF70BE29F63
:102580008001E39F100DF29F100D1124E12F722F97
:102590004230510599F048F44115510569F0413038
:1025A000510581F0EB2F8D2F07C04430510569F0A4
:1025B00080F046305105B1F76E2F8FCFE22F7B2F81
:1025C000812FFACFE22F7D2FF7CFEB2F822F712FA4
:1025D000F3CF7B2F822FED2FEFCF41E00E945A12D5
:1025E000089508950E94ED120895CF93DF93762FFA
:1025F000E901682F842F0E94F212798368838A830D
:10260000DF91CF9108958091C602982F9E7F29F483
:10261000817082608093C60208958635E8F38170E8
:102620008465F8CF88E090E00E9478290895CF92E1
:10263000DF92EF92FF926B017C010E940313B701BE
:10264000A60188E090E00E949629FF90EF90DF902D
:10265000CF900895E6ECF2E083E0808311828FEF63
:1026600082838383148260817181828193810E943D
:10267000171308958091C60280FF02C086950895C1
:1026800080E008959091CA02933018F49F5F909370
:10269000CA02882351F06091C6027091C7028091EE
:1026A000C8029091C9020E941713089581E00E9408
:1026B000421308959091CA02992319F09150909372
:1026C000CA02882351F06091C6027091C7028091BE
:1026D000C8029091C9020E941713089581E00E94D8
:1026E0005A13089570E00E94391A089560910A0102
:1026F0008091C60280FF0BC08091090123E0829F78
:10270000C001112485539D4F0E947213089580913A
:102710000B0190910C0123E0829FF0011124E553FD
:10272000FD4F891748F71182108212828F5F33960E
:10273000F8CF9091C60290FF0EC090910B012091AE
:102740000C0133E0939FF0011124E553FD4F9217E4
:1027500018F00E94761308958183608342839F5FFF
:102760003396F5CFA3E0B0E0E8EBF3E10C94CA2890
:102770009091C60290FF0AC09E012F5F3F4F0E94BA
:10278000F5124B8169818A810E9499132396E2E0B8
:102790000C94E628CF93DF93EC01EC81F0E0EF524C
:1027A000FB4F4491E6ECF2E0628181810E94B2131A
:1027B0008C818F5F8C83DF91CF910895CF93DF93CE
:1027C000EC01E6ECF2E0438162818C810E94B2135D
:1027D0008C818F5F8C83DF91CF910895A3E0B0E06F
:1027E000E4EFF3E10C94C8288C0180913E02811142
:1027F0000AC09E012F5F3F4F4FEF6FEF0E94F5120F
:102800008A8180933E02F8016481613069F0809191
:102810003E0240E0662361F040E0623011F44091F6
:102820003E0280E060E004C060913E0240E080E053
:102830000E949913F801848190E0019663E070E0B2
:102840000E944D2884832396E4E00C94E428A3E0BE
:10285000B0E0EDE2F4E10C94C328082FD62EE42E6C
:10286000C22E9091C60290FF29C0E92FE695AE2FA7
:10287000B0E0A956BE4F8C9180935E029E7F92304D
:1028800009F59E012F5F3F4F802F0E94F5124B816B
:1028900069818A810E9499130093C702D092C8026D
:1028A000E092C902CC2051F06091C6027091C7023B
:1028B0008091C8029091C9020E9417132396E9E003
:1028C0000C94DF28823019F4E090C902E5CF8630FD
:1028D00019F40091C702E0CF8930D9F38931E1F6CC
:1028E000E9516E2F6170B62EE695F0E0EF52FA4F87
:1028F0001491F12C60910D01F61618F00E947613D8
:10290000CBCFF19EC001112470E00E943928802FA6
:10291000B11014C0860F20910B01622F6F0D772725
:10292000771F9B01220F331F260F371F25533D4F63
:102930004E2D6D2D0E94F512F394DCCF861BEBCF4C
:10294000E6ECF2E09181282F438162818AE0890FD1
:102950000E942714089581E00E94A0140895E6ECD7
:10296000F2E09181282F4381628186EF890F0E94D6
:102970002714089581E00E94AF140895E6ECF2E078
:10298000628121E1620F08F46FEF282F438181817A
:102990000E942714089581E00E94BE140895E6EC79
:1029A000F2E0628121E1621B08F460E0282F43819C
:1029B00081810E942714089581E00E94CF14089518
:1029C000E6ECF2E0438121E1420F08F44FEF282FBB
:1029D000628181810E942714089581E00E94E014A1
:1029E0000895E6ECF2E0438121E1421B08F440E067
:1029F000282F628181810E942714089581E00E941E
:102A0000F114089520E00E9427140895EF92FF9298
:102A10001F93CF93DF93EC0110E0EE24EA94F12CA6
:102A200060910D01161770F00E9476139A818C81C7
:102A300090FF27C08F5F8C83DF91CF911F91FF9014
:102A4000EF90089520910B01422F410F5527551FFC
:102A5000CA019A01220F331F280F391F25533D4FFA
:102A600070E0C7010E944D28962F8C814091C902C9
:102A70006091C802199F800D11240E94F5121F5FFA
:102A8000CFCF8150D8CFB0E0A0E0E9E4F5E10C94DD
:102A9000C328FC0182810FEF80FF01E010E08091EC
:102AA0000D01181798F00E947613809140020130B2
:102AB00009F04CC0811102C080910D0181508093BA
:102AC0004002CDB7DEB7E9E00C94DF28C0910B01DE
:102AD000C12ED12CCC0DDD2DD11DCE01880F991F1B
:102AE000C80FD91FC553DD4F198218821A8234E0EE
:102AF000E32EF12CB12C809140028B0D853004F136
:102B00008370082E000C990BC816D90691F4809199
:102B1000C9028E9DA0018F9D500D1124559547959A
:102B2000559547959E016091C8028091C7020E9409
:102B3000F512B00EF1E0EF1AF108E9F61F5FAFCF22
:102B400087FFDFCF90910D01890FDBCF90E00196D9
:102B500060910D0170E00E944D28B1CF0F931F933B
:102B6000CF93DF9380910B0190910C0123E0829F22
:102B7000F0011124E553FD4F891740F1C0E0D3E087
:102B800060910D01C61740F10E9476132091070154
:102B900080913F02820F80933F0290910801920F33
:102BA00090930801191654F4082E000C990B4091CB
:102BB0000D014150550B841795071CF0219520936A
:102BC0000701DF91CF911F910F910895118210821B
:102BD00012828F5F3396D0CF0C2F10E070E0C801C7
:102BE0000E944D2820910B01820F482F50E0209128
:102BF0003F02022E000C330B02171307BCF020918A
:102C00000801022E000C330B201731077CF08D9F3A
:102C10009001112425533D4F4091C9026091C80293
:102C20008091C7020E94F512CF5FAACFFA01EE0F82
:102C3000FF1FE40FF51FE553FD4F11821082128232
:102C4000F3CFB0E0A0E0E7E2F6E10C94C028EC019D
:102C50004C81042F10E09801D8010E9491289B011B
:102C6000AC010E94A7284B015C01E0E2F0E0E01B10
:102C7000F10BA5E5B0E0AC019B010E94A7286B0118
:102C80007C019F01DF010E9489289B01AC010E9409
:102C9000B2289B01AC01280D391D4A1D5B1DC701DF
:102CA000B6010E946128F22E822F90E039E23F1592
:102CB00020F143E0249F9001112435952795122F90
:102CC000109500E085E5E82EEF1880910D010817BA
:102CD00018F10E9476139C8181E0992319F09032BB
:102CE00019F48FEF8093060180910601890F8C8380
:102CF000CDB7DEB7ECE00C94DC2825E530E0B90177
:102D0000681B790B9B01220F331F260F371F37FFDC
:102D1000D4CF2F5F3F4FD1CF8E2D01FD8F2D20912E
:102D20000B01622F600F7727771F9B01220F331F44
:102D3000260F371F25533D4F412F6091C8020E9437
:102D4000F5120F5FC2CF0F931F93CF93DF93EC0168
:102D500010E000E090910D019017110609F06CF45D
:102D60000E9476138C8190E00196817099278C8364
:102D7000DF91CF911F910F91089520910B01A80130
:102D8000420F511D9A01220F331F240F351F255367
:102D90003D4F4C816091C8028091C7029695901773
:102DA000110651F04CF0442349F04091C9020E94B1
:102DB000F5120F5F1F4FCECF4423B9F340E0F7CF9A
:102DC000B0E0A0E0E6EEF6E10C94BC28FC016280E5
:102DD000448081E08483E1EDF4E07490E0E5F5E087
:102DE000E491812C75E0972EF2E0CF2EDD24D39470
:102DF000AA24AA94B12C55245A94E7190E2F10E056
:102E000080910D01881638F00E947613CDB7DEB799
:102E1000E0E10C94D828E82CF12C82E0861568F0CB
:102E20009E9CF0019F9CF00D1124EF5BFD4F809163
:102E3000C70280838091C8028183411023C09E9C79
:102E4000F0019F9CF00D1124EF5BFD4F1382128265
:102E500020910B01C701820F911D9C01220F331F8E
:102E6000280F391F25533D4F9E9CF0019F9CF00D6C
:102E70001124EF5BFD4F4281618180810E94F51238
:102E80008394BECF9E9CE0019F9CD00D1124CF5B0C
:102E9000DD4F8B818823E9F081508B83859DC001B4
:102EA00011246C8170E00E943928FB01FF27EF524A
:102EB000FB4F8491E82FE719E59DC0011124B8016B
:102EC0000E9439288091C902689FB00111247A8339
:102ED000BFCF0E943D292091C902269521582C9DE3
:102EE000A0012D9D500D1124452F552784179507BE
:102EF0000CF0AECF82E0861588F40E943D29B50122
:102F00000E944D2888830E943D292091C802269561
:102F1000622F70E00E944D28280F29839E9CF001AB
:102F20009F9CF00D1124EF5BFD4F12828091C9022E
:102F3000893C58F088EC9E9CF0019F9CF00D112478
:102F4000EF5BFD4F8483838383CF8431A0F784E1DB
:102F5000F2CFE6ECF2E080818E7F80836081718128
:102F6000828193810E94171310925F022FEF80E7F6
:102F700092E0215080409040E1F700C000000E94A4
:102F800076130895E6ECF2E080818E7F80831092C4
:102F90005F022FEF80E792E0215080409040E1F700
:102FA00000C000000E947613089510925F02809185
:102FB0005C0281110AC081E080935C028091C602AC
:102FC000817080935B020E94C21708956091C602CF
:102FD000669570E04BE050E08EE091E00E944D2954
:102FE000892B19F481E080935F020E94292190933C
:102FF00056028093550208959091C60290FF2BC00F
:103000009170811129C092609093C602662351F09D
:103010006091C6027091C7028091C8029091C90266
:103020000E9417136091C602669570E04BE050E075
:103030008EE091E00E944D29892BA9F010925F0249
:1030400081E0809358024091C9026091C80280914A
:10305000C7020E94021508958B3210F09465D4CFF8
:10306000880F982BD1CF0E94E617EACF682F909156
:10307000C602969581E0890F8B3208F081E00E94AC
:10308000FC17089581E00E9436180895682F9091EA
:10309000C60296958FEF890F09F48AE20E94FC1709
:1030A000089581E00E944618089561E00E94FC178F
:1030B0000895E6ECF2E080818160808386950E942D
:1030C000551808958091C60280FF03C00E94A91779
:1030D00008950E945918089560E00E94FC17089511
:1030E00080915D0281112EC00E94B40D811104C037
:1030F0000E945D0E0E942A130E9412136093C60262
:103100007093C7028093C8029093C9026E7F61F4E6
:103110000E942A130E9412136093C6027093C70282
:103120008093C8029093C9020E94031310925F0219
:103130008091C60280FF03C086950E946C1881E0D2
:1031400080935D020895E6ECF2E0808181608083E7
:1031500086950E946C18089510925C0280915B0223
:1031600081110E94A3180E94E61708950F931F93E0
:10317000CF93DF9380915F028823B9F180915E0243
:10318000E091C602E695E81BE0935702823091F584
:10319000F0E0E353FB4FE491CE2FD0E00AEC13E1D3
:1031A00080915802882361F0109258020E942921D0
:1031B000909356028093550210925A02109259022F
:1031C0000E942921E0915502F09156028E1B9F0B1F
:1031D0008F3F9F4750F4EC0FFD1FF0935602E09392
:1031E000550285E592E0F8010995DF91CF911F9195
:1031F0000F910895863049F4F0E0E653FB4FE491D7
:10320000CE2FD0E00EED13E1CBCF893051F4E6950F
:10321000F0E0E953FB4FE491CE2FD0E006E015E15A
:10322000BFCF8F3051F4E695F0E0EC53FB4FE491C3
:10323000CE2FD0E003E415E1B3CF853149F4F0E0BF
:10324000EF53FB4FE491CE2FD0E00EEA15E1A8CF6B
:10325000C8E2D0E001E216E1883109F4A1CF83325F
:1032600039F4EFEBF4E0C591D4910EEE13E198CF71
:10327000C4EFD1E003EA16E1843209F491CFC0ED46
:10328000D7E001EF12E1853209F08ACF8E2F63E09B
:103290000E942D28E92FF0E0E454FB4FE491CE2F5B
:1032A000D0E000EE16E17CCFFA01811101C0FB01F4
:1032B00009950895CF93DF93C82FD62F0E943A1314
:1032C0008C1748F00E943A138D1728F40E94421878
:1032D000DF91CF9108958C2F0E945518F9CF1F933D
:1032E000CF93DF93EC01FB01128111111BC00E94EF
:1032F000C60C8272CD3CFCE5DF0709F4A0C008F0E3
:1033000045C0C73CECE5DE0709F485C0F8F4C43CD1
:103310009CE5D90709F475C050F4C33CDC4509F4B9
:103320006DC011E0812FDF91CF911F910895C53CB1
:103330009CE5D90709F46AC04AEB54E16BEA74E1F1
:10334000C63CDC4571F70E945419ECCFCA3CFCE541
:10335000DF0709F46AC068F4C83CECE5DE0709F44D
:103360005FC04BEC54E16CED74E1C93CDC4559F3B2
:10337000D8CFCB3C9CE5D90709F45CC04EE653E1BD
:1033800066E573E1CC3CDC45F1F2CBCFC23DFCE518
:10339000DF0709F463C098F4CF3C9CE5D90709F432
:1033A00057C008F451C0C03DFCE5DF0709F453C025
:1033B000C13DDC4509F0B5CF6EE089E01CC0C53DDC
:1033C0009CE5D90709F450C058F4C33DFCE5DF077C
:1033D00009F447C0C43DDC4509F0A3CF88E135C0FE
:1033E000C63D9CE5D90709F442C06AE285E2CE35C4
:1033F000DD4509F096CF0E945A1994CF0E946218B9
:1034000091CF41E558E162E478E19DCF42E458E193
:1034100061E578E198CF4BEA54E16AEB74E193CF30
:103420004CED54E16BEC74E18ECF4EEF54E16DEE58
:1034300074E189CF4DEE54E16EEF74E184CF46E53F
:1034400053E16EE673E17FCF81E00E9455186ACFA9
:1034500065E082E0D0CF68E086E0CDCF64E18FE028
:10346000CACF67E185E1C7CF62E289E1C4CF83E2D9
:10347000ECCF539A4BB1477F5BB15860EFB7F894EC
:103480009B01220F331F260F371F280F391F2817C4
:10349000390741F4EFBF8FE594E00197F1F700C0E1
:1034A00000000895DC016D91CD0178E05BB900006A
:1034B00000C067FF4BB9660F000000C000C000C02D
:1034C0004BB900C07A9591F7E2CFB0E0A0E0EBE60F
:1034D000FAE10C94C4286C017B0164E670E088E793
:1034E0000E94FA1EEC0197FD12C010E000E0F60108
:1034F000E00FF11F849164E670E00E94661FEC010A
:10350000892B29F40F5F1F4F0E151F0581F70E94AD
:10351000DC1FCE01CDB7DEB7E8E00C94E0280895BB
:10352000E7EDF2E080E094E0DF019C011D92215084
:103530003040E1F7F093DC06E093DB068FEF9FEF7E
:103540009093A6028093A50208950E948F1A0E946C
:1035500017048093A10280FD0FC080E88093A00231
:103560000E94F41E6DE070E08DEE96E00E94651AF8
:10357000892B21F080E0089580E4F0CF8091A102B2
:1035800063E070E081FD26C08AEE96E00E94651A35
:10359000892B81F76DE070E08AED96E00E94651A54
:1035A000892B41F70E943521605E714B8F4F9F4FF1
:1035B0006093D7067093D8068093D9069093DA0665
:1035C0000E94901A81E08093A4028093A30210923B
:1035D000A202089587EE96E0D9CF2091A00236E0AE
:1035E000839FC0011124629F800D911D11248115BC
:1035F00024E0920714F090E080E089529D4F909370
:10360000DC068093DB060895CF93DF932091DB06E1
:103610003091DC06275D3240A901460F571F41302B
:10362000544020F060E074E0621B730B4091A502EF
:103630005091A602FC01C901620F731FC1E0D0E0E6
:103640008617970738F05093A6024093A502DF91A2
:10365000CF9108952491DC01A952BD4F3C913217BE
:1036600081F02C939C01A6E036952795AA95E1F769
:10367000DE0102C0AA0FBB1F2A95E2F79D014A2B6B
:10368000532B01963196DCCF8091A402811103C0A7
:103690008091A30208950E943521605E714B8F4F87
:1036A0009F4F6093D7067093D8068093D906909366
:1036B000DA068091A3028111EBCF62E070E088ED21
:1036C00096E00E94651A892B19F781E08093A30286
:1036D000DFCF2F923F925F926F927F928F929F9255
:1036E000AF92BF92CF92DF92EF92FF920F931F9310
:1036F000CF93DF938091A402882369F02091A502E3
:103700003091A6022115310531F08091A20261E0CD
:1037100070E0882399F0DF91CF911F910F91FF9076
:10372000EF90DF90CF90BF90AF909F908F907F9061
:103730006F905F903F902F9008958F5F082F10E05B
:103740001B01082E02C0220C331C0A94E2F7A901C7
:1037500042215321452B89F39091A10290FD43C052
:103760008295880F880F807480931B01980136958D
:10377000279520931E01815C80931C0110921F01EC
:1037800024E630E047E050E069E171E088E70E941C
:10379000941F892B09F0BFCFA80126E0440F551FC5
:1037A0002A95E1F78091A10280FD2BC049525D4F1F
:1037B00004E610E020E430E060E488E70E94B51FF2
:1037C000892B09F0A8CF0E94441BE101C095D09538
:1037D0008091A5029091A602C823D923D093A60276
:1037E000C093A50298CF880F880F880F80931B0184
:1037F00010921E01895F80931C0187E080931F0156
:10380000BFCFE0E6F2E080E4DF011D928A95E9F7A0
:10381000AAECB1E002EC11E082EDC82E81E0D82ED6
:1038200097E0592E772473948D91E80129918E01A8
:10383000240F352F311D29523D4FE82FF0E0E05A7B
:10384000FD4F90E080E0652C681A872C082E01C09F
:10385000880C0A94EAF77901A12CE701B9907E015E
:10386000B820662D6A196770962E062E000C770B0D
:10387000DB2D01C0DD0F9A94EAF77195619571090E
:103880006770772701C0B6946A95EAF7BD2A608110
:10389000962E9B289082A39468E0A612DECF019614
:1038A00031968830910579F6CA16DB0609F0BCCF4F
:1038B00004E610E020E430E040E652E07DCF809165
:1038C000A3029091A402911103C091E08927089569
:1038D000882369F062E070E086ED96E00E94651A48
:1038E000892B19F08091A30208951092A302809170
:1038F000A302EBCF81E008950F931F938091A40260
:10390000882309F160E080E00E94ED1A0E9419040A
:103910000E94691B8091A3028823A9F00E9435218F
:103920000091D7061091D8062091D9063091DA0679
:10393000601B710B820B930B6F3F7F4F8F4F9F4725
:1039400010F40E945F1C1F910F910895CF93DF9395
:10395000EC01FB018281882309F464C1C430FDE5D8
:10396000DF07E0F5CB3F9CE5D90730F49E012250FC
:103970003C4524313105D8F50E94C90D9093C10210
:103980008093C002C231ECE5DE0709F41FC108F0E4
:103990006EC0C9308CE5D80709F4F2C008F03FC00A
:1039A000C530ECE5DE0709F4DBC058F5C3308CE523
:1039B000D80709F4CDC008F0CFC08091C002816063
:1039C000C230DC4509F4AEC08091C0029091C102C2
:1039D0000E94D70D0E944B0880E009C0C63AEDE571
:1039E000DE0751F238F4C2369DE5D90729F2DF919E
:1039F000CF9108959E012E5A3D4523303105B8F7E9
:103A0000BBCF8091C0028062C730FCE5DF0709F4BC
:103A100089C008F4B1C08091C002806483C0CD30F9
:103A20009CE5D90709F4BAC070F48091C0028E7F7A
:103A3000CB30FCE5DF0709F475C008F4A7C080911E
:103A4000C0028D7F6FC0CF309CE5D90709F4B6C0A6
:103A500008F4A8C0C031FCE5DF0709F4B3C0C131E8
:103A6000DC4509F0B1CF8091C0028F7B5BC0C115EE
:103A70009DE5D90709F4B4C098F5CB3FFCE5DF0715
:103A800009F472C0B8F4C4319CE5D90709F4B6C092
:103A900008F4A2C0C531DC4509F096CF8091C00280
:103AA00082FB992790F921E0922790FB82F990FB05
:103AB00083F938C0CD3F8CE5D80709F477C008F406
:103AC00057C0CE3FECE5DE0709F474C08091C10217
:103AD0008360CF3FDC4509F077CF8093C10274CF7C
:103AE000C2368DE5D80709F496C068F4C230EDE51A
:103AF000DE0709F48CC008F477C0C330DD4509F057
:103B000063CF80E085C0CE3A9DE5D907E9F068F43F
:103B10009091C002892F8E7F90FF8160C63ADD456B
:103B200009F052CF8093C0024FCFCF3A8DE5D8072E
:103B300089F1C03BDD4509F047CF9091C102892F43
:103B4000877F93FF8860C9CF8091C1028860C5CF0D
:103B50008091C0028260E6CF8091C0028460E2CF93
:103B60008091C0028860DECF8091C1028160B5CFB4
:103B70008091C1028260B1CF8091C0028061D2CFBA
:103B80000E944B088091C0028068CCCF8091C00217
:103B90008C60C8CF8091C102877F9FCF8091C00287
:103BA0008B7FC0CF8091C002877FBCCF8091C10244
:103BB0008E7F93CF8091C1028D7F8FCF8091C00285
:103BC0008F7EB0CF8091C0028F7DACCF0E944B081A
:103BD0008091C0028F77A6CF8091C002837FA2CF51
:103BE0008091C1028C7F79CF8091C102982F9095EE
:103BF00091708E7F892B90FB81F96FCF0E944B08CB
:103C00009091C002892F97FB87F980588BCF81E074
:103C10000E94600ED9CE9091C002892F8F7E94FFB2
:103C2000806180CF81E0E3CECF93DF93EB018631DB
:103C30009C4511F50E94C60C9A81992399F08A7AC5
:103C400091E009F490E09093A702811109C089E204
:103C50000E949E0C0E94070D80E0DF91CF91089595
:103C600085E3F6CF8091A702811104C089E20E940A
:103C7000A60CF0CF85E3FBCF81E0EFCF0F931F932E
:103C8000CF93DF93C42FD22FFC0182818823C9F008
:103C90004093AA020E9429219093A9028093A8022E
:103CA00080E28C0F883040F4C77081E001C0880F3B
:103CB000CA95EAF70E94FC05DF91CF911F910F9101
:103CC00008951091AA02141332C08091A802909115
:103CD000A9020E944121883C910548F5C0E2CD0F20
:103CE0001D17B9F080E2810F883040F4177081E031
:103CF00001C0880F1A95EAF70E940306C83048F4FD
:103D000081E09D2F977001C0880F9A95EAF70E9475
:103D1000FC05802F0E94F305C83070F6D77081E053
:103D200001C0880FDA95EAF70E940306C5CF80E24A
:103D30008C0F883008F6C77081E001C0880FCA95E3
:103D4000EAF7F2CF0F939C01CB01243F4CE53407F7
:103D500059F1A8F4293DFCE53F0701F12A3D4CE566
:103D60003407D1F1283D3C4591F406E221EE41EEC5
:103D700068ED7CE50E943E1E80E00F910895263F8D
:103D8000FCE53F07E9F0B0F0273F3C45F9F0FC01C6
:103D90008281882339F11092AA02EFCF07E225EE43
:103DA00045EE69ED7CE5E6CF06E221EE40EE64EFFC
:103DB0007CE5E0CF07E225EE44EE65EF7CE5DACF67
:103DC00006E221EE42EE66EF7CE5D4CF07E225EE77
:103DD00046EE67EF7CE5CECF08E221E045EE6AEDE6
:103DE0007CE5C8CF81E0C9CF1092B9008CE0809308
:103DF000B8000895B0E0A0E0E0E0FFE10C94C12835
:103E0000B82EEB010E9429216C01EE24E394F12CE1
:103E1000C431D10560F025E0E22EF12CCF3FDC0764
:103E200031F0CE0164E170E00E9439287B0184EA20
:103E3000A82E94E8992E1092BC00A092BC000E947B
:103E400029218C018091BC0087FF0DC08091B900B1
:103E5000887F8830F9F08091B900887F8031D1F077
:103E60000FEF1FEF08C0C8010E944121E816F906B4
:103E700048F70EEF1FEFCF3FDC07E9F2C6010E94C3
